:030000000219FDE5
:03000B000200A848
:03002B0002015A75
:03005B000202EBB3
:030073000202D8AE
:1000800002030406080C10182030406080040608A3
:100090000C10182030406080A0C00003070F1F051F
:1000A000050D050305030302C2AFC0D0C0E0206206
:1000B00014E5256009E473E525F4F58AD262D0E001
:1000C000D0D0D2AF3285268AC262E526F4602F30C6
:1000D000682520720DD0E0D0D0D292D291D290D2A9
:1000E000AF32D292D291D290206F0C206509740A5F
:1000F000D5E0FDE57B4290D0E0D0D0D2AF32758A1A
:1001000000C28DD26201F701B7306805206502C2D6
:100110009201B7306805206502C29101B7306805C9
:10012000206502C29001B7C29330680A2065077447
:1001300008D5E0FDC29201B7C29430680A20650775
:100140007408D5E0FDC29101B7C29530680A2065F8
:10015000077408D5E0FDC29001B7C2AFC2AD53E647
:10016000EFC0D0C0E0D2D3D2AFC2CEE52A60072024
:10017000744F152A21C17800790020742EE5803053
:100180007E01F430E40278FF53DACF207E0343DAB5
:1001900020307E0343DA10C2D8C271E580307E0180
:1001A000F430E40279FFC3E89970CB306103752A1B
:1001B00018207403752A18885CD270E86003755F94
:1001C0000020740DE52B6004152B21D143DA01C208
:1001D000D82070024144A85C206102C270207431B2
:1001E000C3E894F0400374F0F8E8C4540F28F87999
:1001F00084B703024111C313C3138721200802C32C
:1002000013200A06C3C898F8411128F8500374FF58
:10021000F8C3E895655003E565F88822E52D540696
:100220006022206B1FE536C333C333F8E564C31384
:10023000C313F9C3952240028922E82522F52250F2
:10024000037522FF852224A824C3E524956140027A
:10025000A8618825E56670024188C3E8AA669A50BD
:1002600003E8FAE4F9EAC333FBE568F45B29400DDF
:100270002567F8E56760021567400B41880AC3E50A
:10028000679A5002056778FF8826C26FC3E52694F7
:10029000F84002D26F20CF0AD0E0D0D043E610D28F
:1002A000AD32C2CF053A7801E52A600530740215F7
:1002B0002AC3E55C94014005755F0041CE7560007E
:1002C000756900E55F2401F55F5003755FFFD0E0BD
:1002D000D0D043E610D2AD32C2AF53E67F7592FA6A
:1002E0007593FFC260759104D2AF32C2AF53E6EF8F
:1002F000C2ADC0D0C0E0C0F0D2D3D2AFA8FBA9FC41
:10030000C2D8307102615253DACF207E0343DA1033
:10031000307E0343DA20D271E580307E01F420E4A0
:1003200002612988278928A17F53DACF207E0343E1
:10033000DA20307E0343DA10C2D8C271307402A1D1
:100340006B7800E580307E01F430E402A16B885CBC
:10035000A15353DACF207E0343DA20307E0343DA01
:1003600010C271206102812B53DACF207E0343DA61
:1003700010307E0343DA20C2D8D27188578958C31F
:10038000E89555F8E99556F97B007E087A00C3E8B0
:10039000948CE994005005755B00811D882178A23A
:1003A000E6A8216055C3E894C8E994005008E4D257
:1003B000E4FB7A0A61F8C3E89468E994015008E420
:1003C000D2E3FB7A0F61F8C3E894D0E994025008B5
:1003D000E4D2E2FB7A1E61F8C3E894A0E9940550E8
:1003E00008E4D2E1FB7A3C61F8C3E89498E9940808
:1003F0005008E4D2E0FB7A787E00C3E89559FCE926
:10040000955AFD30E70AECF42401FCEDF43400FDCC
:10041000755B00C3EC9AED9E5003755B01885989AA
:100420005A8557558558567802A153C3E89527F841
:10043000E99528F9307C02A137307B02A137307A68
:1004400002A130207502814EE9FDE8FC816DE9C30F
:1004500013F9E813F8307902A130E9C313F9E8136E
:10046000F8307802A130E9C313FDE813FC20612CB9
:0F047000C3EC941CED940240028184ED701EC316
:10047F00EC94C850180529E52970021529C3E52900
:10048F00940A5002A16B755C00D270A16BE52960D4
:10049F000215297888E6F97400207F087896B90349
:1004AF0002789EE624FAFEE43400FFC3EC9EFCEDD6
:1004BF009FFD9208B90310A2085007207609D27643
:1004CF0081D6307602C276A2085016B9030DECF42D
:1004DF002401FCEDF43400FD0204F078007900A152
:1004EF0037B90315EC33FCED33FDC3EC940AFCED87
:1004FF009400FD50047C007D00C3EC94FFED94004C
:10050F00400678FF7900A137EC8572F0A4C5F0A200
:10051F00F733F87900400302055378FF790002059D
:10052F0053E9C313F9E813F8307C0EE9600278FF42
:10053F00C3E81338F8E43400F9C3E894FFE99400F2
:10054F00400278FF885CD270206102A16B741FF4A7
:10055F00552F4BF52FC274EB7002D274752A1830D9
:10056F007403752A0A306102A17F20740353DAFEE7
:10057F00207403752B06D0F0D0E0D0D0D2AD43E677
:10058F00103279010205AF79030205AF790A02052E
:10059F00AF791E0205AF79640205AF79C80205AFC6
:1005AF007817E4D5E0FDD8FAD9F6227A147B7802D1
:1005BF0005D67A107B8C0205D67A0D7BB40205D650
:1005CF007A0B7BC80205D6E573D5E001227902E4E8
:1005DF00C294D5E0FDC291D5E0FDD291D5E0FDD218
:1005EF0094D5E0FDE920E002C29230E002C290E52E
:1005FF0073D5E0FDE920E002D29230E002D2907490
:10060F0096D5E0FDD9C9EAF8D5E0FDD8FBDBB8C235
:10061F009422C37C007D0075F00005F0EA33FAEBFD
:10062F0033FB50F6EB13FBEA13FAC3E9FFE8FEE8DE
:10063F009AF8E99BF95004EFF9EEF8B3EC33FCEDBF
:10064F0033FDD5F0DFEDF9ECF822E889F08A20D2FE
:10065F00D4F8A9F07B0030F70B7BFFF42401F8E905
:10066F00F43400F9E88520F0A4ADF0F8E98520F026
:10067F00A4AFF0FEED2EF974003FFA7C04C3EA1329
:10068F00FAE913F9E813F8DCF48BF030F70AE8F421
:10069F002401F8E9F43400F9E889F0C2D4F8A9F09C
:1006AF002222C3E54113F9E54013F8C3E54498F856
:1006BF00E54599F9500CC3E89480E994FF40160280
:1006CF0006E8C3E8947FE9940050030206E8787FB8
:1006DF0079000206E8788079FF8849894A22E5493E
:1006EF002546F8E54A3547F9854A20E4300701F4F5
:1006FF003548FA30E709C3EA94F04015020726C3DC
:10070F00EA940F500302072678FF79FF7A0F02074A
:10071F0026780079007AF0C3E5249561500AC374F6
:10072F00019524500B020744E54A20E70E020744C7
:10073F00E54A30E706884689478A482278A5E6FACF
:10074F00C3E54933F8E54A33F9D159E930E70BC32B
:10075F00E89480E994FF4013E17EC3E8947FE99425
:10076F00005002E17E787F7900E17E788079FFE8A2
:10077F0020E715C3E52398F84009C3E89401400327
:10078F000207A578010207A5E8F424012523F84004
:10079F00030207A578FF884B2278A6E6FAA847A997
:1007AF0048D159E930E70CC3E89401E994FF4016AA
:1007BF000207D9C3E894FFE9940050030207D978E0
:1007CF00FF79000207D9780179FFE920E715C3E522
:1007DF004B98F84009C3E8940140030208007801E0
:1007EF00020800E8F42401254BF8400302080078C2
:1007FF00FF88242278FF20692879A1E76023E5414B
:10080F00601F74FF8541F0848539F0306A0375F0FD
:10081F0005A4F8C5F0600278FFC3E895645002A8FC
:10082F0064886322C3E5409440E5419401E5635039
:10083F0003140144046002F5632202084C2275E898
:10084F0090227883E6FF30EDF9A8BDA9BE0570C3ED
:10085F00E57094084052757000E9FA79A0E760449A
:0E086F00EA7007E571601B020885C3E8957109
:10087D006010E5715006600C140208910460F902D5
:10088D000891E571F571C39458401B7561C0C3940F
:10089D00044013756180C39404400B756140C3948B
:1008AD0004400375610075BB0322E561F460020528
:1008BD0061E570B4070375BB1022743279A787F018
:1008CD00A4C5F0A2F733F8C3E895614002A861888A
:1008DD00228824882588268864227540007541F079
:1008ED0022C2AF75C820A8CCA9CDAA3A30CF010A33
:1008FD0075C824D2AFAB3BAC3C883B893CC3E89B6D
:10090D00F8E99C206908F930660221FF2159AD3DB7
:10091D008A3DF9EA9DFA600678FF79FF213EAE3EE9
:10092D00AF3F8B3E8C3FA83BA93CC3E89EF8E99FA7
:10093D00F9C3E54113FBE54013FAE82AF540E93B1D
:10094D00F54150067540FF7541FF21A6AA40AB4108
:10095D00AC40AD417E047F02C3EB9404400D1E1FDD
:10096D00C3EB94084005206A021E1FC3ED13FDEC76
:10097D0013FCDEF7C3EA9CFAEB9DFBEF6009C3E9BC
:10098D0013F9E813F8DFF7EA28FAEB39FB8A408B05
:10099D004150067BFF8B408B41C3EB94025002D23A
:1009AD00663069047F0321D17892E6FFC3E5379461
:1009BD008240110FC3E53794A040010FC3EF940699
:1009CD0040027F057E02E541C4540FF9E541C45450
:1009DD00F0F8E540C4540F28F8C3E89EFAE99400F6
:1009ED00FB4009C3EA9402EB940050047A02E4FB45
:1009FD00414BAA40AB41EBC4FEEAC4540F4EFCC3BD
:100A0D00EA9CFAEB9400FBC3E813C313F8EA28FA47
:100A1D00EB3400FB8A408B41C3EB94024002C2666B
:100A2D007802EBC4FE7B00EAC4540F4EFAC3EA9879
:100A3D00FA4005C3940250027A027892E6FF3060C4
:100A4D0002414B855192855293D26043E680C3E4B7
:100A5D009AF8E49BF930660241D7E8FAE9FBD3E94D
:100A6D0013FDE813FC88518952C3EF94036038EFEE
:100A7D0020E00DE82CF8E93DF9ECFAEDFB020AA0B7
:100A8D00E828F8E939F9C3E82402F8E93400F97ADD
:100A9D00FE7BFFC3EF9403400E8A538B54884D8920
:100AAD004E8C4F8D50610B885389548A4D8B4E8CD3
:100ABD004F8D503069127553F07554FF754FF075A9
:100ACD0050FF7551F07552FF610BE8FAD3E813FC36
:100ADD008851C3EF94036020EF20E007E82CF8EC79
:100AED00FA41F7E8282402F87AFEC3EF9403400890
:100AFD008A53884D8C4F610B88538A4D8C4FE56816
:100B0D00C3335002646BF5683060026115753402B1
:100B1D00D26043E680E52D54066034A840A941C358
:100B2D00E913F9E813F8C3E913F9E813F830690488
:100B3D00E92440F9C2AF53E67F759100C3E498F5FF
:100B4D0094E499F595759104D26043E680D2AF2275
:100B5D00D264754300752000306C03752040020B84
:100B6D007CD264754300752040306C03752000788D
:100B7D00017901206620E52D54066002C2647914C6
:100B8D00E541C313700104F8C39414400278143086
:100B9D006904781B791B206010E543600C306903F4
:100BAD00D53404D26D8127711D0543E59BF4544066
:100BBD00B52002811130690908C3E8994001186117
:100BCD00A320640A08C3E8994002617C61A3C26452
:100BDD00C2AF53E67F75910030661275940075951E
:100BED00F8759104D26043E680D2AF617CE5417E19
:100BFD00FFC3334005C3334001FEC3E49E7594002B
:100C0D00F59561EEC3E53394015002617C306402C9
:100C1D00617CD802812561A3C26DC2AF53E67F7599
:100C2D009100855394855495759104854D92854E0B
:100C3D0093D26043E680D2AFE52D54066008206A5A
:100C4D00020533020C63306D0D206C0A206407150C
:100C5D008115810215412278003064027801E53753
:0E0C6D0075F007A4F9E5F028F5F0E9A2F01300
:100C7B00A2F113A2F213F537C394785003753778AA
:100C8B00C3E53795384008D265D292D291D29030D5
:100C9B006002819A854F92855093D26043E6802201
:100CAB00D2A0207D16C2AF754202C294D29330629D
:100CBB0002C290D2AF759F10020EA7C2AF7542024F
:100CCB00C294D295306202C292D2AF759F10020EBF
:100CDB00A7C2A0307243207D20C2AF7542039001A2
:100CEB0038757B10D290C295306204C29181FCD2D0
:100CFB0094D2AF759F20020EA7C2AF75420390012D
:100D0B0038757B10D292C293306204C291A11CD26F
:100D1B0094D2AF759F00020EA7207D17C2AF75420C
:100D2B0003900113D290306202C291D2AF759F2013
:100D3B00020EA7C2AF754203900113D2923062022A
:100D4B00C291D2AF759F00020EA7D2A0207D16C212
:100D5B00AF754204C293D295306202C291D2AF7585
:100D6B009F00020EA7C2AF754204C295D2933062A8
:100D7B0002C291D2AF759F20020EA7C2A030724360
:100D8B00207D20C2AF754205900127757B08D2915B
:100D9B00C294306204C292A1A6D293D2AF759F10B7
:100DAB00020EA7C2AF754205900149757B20D29107
:100DBB00C294306204C290A1C6D295D2AF759F1077
:100DCB00020EA7207D17C2AF754205900109D29183
:100DDB00306202C292D2AF759F10020EA7C2AF75DE
:100DEB00420590011DD2913062EBC290D2AF759F3C
:100DFB0010020EA7D2A0207D16C2AF754206C29577
:100E0B00D294306202C292D2AF759F20020EA7C25B
:100E1B00AF754206C293D294306202C290D2AF75C4
:100E2B009F00020EA7C2A0307244207D20C2AF7576
:100E3B004201900149757B20D292C293306204C269
:100E4B0090C150D295D2AF759F00020EA7C2AF755D
:100E5B004201900127757B08D290C295306205C282
:100E6B0092020E71D293D2AF759F20020EA7207DF6
:100E7B0017C2AF75420190011DD292306202C2902F
:100E8B00D2AF759F00020EA7C2AF75420190010948
:100E9B00D290306202C292D2AF759F20C26522906F
:100EAB000107757B00D292D291D290C293C294C2A9
:100EBB0095C26222788076FF0876FF0876FF087667
:100ECB00FF08760308760408760A0876030876018D
:100EDB00087601788C76010876FF0876FF0876FF96
:100EEB000876FF0876FF0876030876FF0876FF087A
:100EFB0076FF0876250876D00876FA0876FA087613
:100F0B00040876FF08760108760008767A0876FFE3
:100F1B000876010876010876000876030876002229
:100F2B007887E6FFC272BF0302D2727888E6C39459
:100F3B00036008C27DE630E102D27DC27E7889E68D
:100F4B0030E102D27EC3EF94026008758E01D2733A
:100F5B00020F63758E00C273227880E614900080B6
:100F6B009378A5F67881E6149000809378A6F678AE
:100F7B0086E61490008D9378A7F67886E6F539C34C
:100F8B0094025003753902789CE67538FFB402035E
:100F9B007538A0B4030375388278A3E61490009AD1
:100FAB0093F566D1AA22227896E6FA7897E6FB7833
:100FBB0088E6B40305C3EB940EFB307F047A007B09
:100FCB00FFC3EB9AFCC3948250027C8275720005BE
:100FDB0072EC8572F0A4C3E5F0947D40F222D27FCF
:100FEB00F1B21205A01205A07A007B007C1012054D
:100FFB0096E55C2AFA74003BFBDCF37C04C3EB1331
:10100B00FBEA13FADCF7FEC27F120FB222757C00EB
:10101B00757D00E5EF20E6037520000520903FFF6E
:10102B00E520146006901DFF1460009304600375A7
:10103B00EF1653D9BF7581C043FF8012059175EF31
:10104B000643B203E5B3240220E70DF521E5E320C7
:10105B00E0068521B343E301120EAA7580FF75A448
:0D106B000075F1D475D4EF75908775A54020
:1010780075F2FF75D5BF75A60175E24275DB467539
:10108800EA02120EAAE4F8F6D8FD756801120EBF3E
:1010980012159278988673753001C2AF1205AA129C
:1010A80005BA1205A01205C11205A01205C812053D
:1010B800A01216BB1205AA1205AA1205A5C2AF7581
:1010C8007C00757D0078FA79FA308407D9FBD8F767
:1010D800021C00120F2B120F64120FB1120FB278FC
:1010E800988673120EAA75881075890275C82475BA
:1010F800910475D84075A82275B80275E690759B5D
:1011080080759D0075D10E75BC5875BB0375BA11F5
:1011180075E880120591D2AF12084975360053DA86
:10112800CF207E0343DA20307E0343DA1043DA010E
:10113800C2D8C2711205AAD2617B037A0CE55B7032
:10114800077A0CDB030210C51205A02070030210F9
:10115800C5C270E55CC3940240E1E52F541F855E6B
:101168005DF55EB55DD5DAD5C26153DACF207E0371
:1011780043DA20307E0343DA10C2D8C27178A2E67F
:101188007008D274E52F54E0F52FC2757529001246
:1011980005A5307409C3E529940A4002D2751205E1
:1011A8009678023074027800C3E55C9840F0C2AFCC
:1011B8001205BA1205BA1205BAD2AF1205AA754CB1
:1011C800007888E6B4030241C5120596788CE6C318
:1011D800940150030212C5E530C394015003021272
:1011E800C5757CA5757DF1207435C3E55C94FF5009
:1011F800030212C5C2AF1205CFD2AF1205A5C3E5CF
:101208005C940150EFC2AF1205BA12059B1205BAE1
:10121800D2AF1205A5C3E55C94FF40E90217407FF1
:1012280005D27F120FB21205A5C2AFC27F120FB24C
:10123800AE5CC3E55C947FD2AF500241D5120591F4
:10124800C2AF1205CFD2AFDFD8120FE9C3EE9405B3
:101258007897F61205AA1216C37F0AD27F120FB228
:101268001205A5C2AFC27F120FB2AE5CC3E55C9493
:101278007FD2AF50E4120591C2AF1205BA12059B96
:101288001205BAD2AFDFD4120FE9EE24037896F62E
:10129800F87997E7C394824003985006E824827847
:1012A80097F61205AA1215E01216F21205A5120FEA
:1012B800B2C3E55C94FF500221E9021740757C0037
:1012C800757D00C3E55C954C4003855C4C1205A513
:1012D80078017988E7B403027805C3E55C98400291
:1012E80021C9C2AF1205CF1205CF1205CFD2AF1256
:1012F80005AA753000E4F531F5320531E531F470B1
:101308003F0532789AE67819146012783214600D25
:10131800787D14600878FA146003753200C3E532EA
:1013280098401D120EAA1205911532753100789950
:101338008673C2AF1205CFD2AF789886731205A50F
:1013480012059BE52A700530740201C578012074E6
:10135800027806C3E55C9840A17888E6C3940360E8
:10136800031205A5E52A70030210C5C2AF120EAA22
:10137800E4F522F523F524F525F526F567D2AF78AF
:1013880085E6C333F565E4F544F545F546F547F5D7
:1013980048F570F52CF52DF53775700875BB1012EA
:1013A800059112084D30EDFDA8BDA9BEE97001F800
:1013B800887112085175700875BB10120F2BC2AFD7
:1013C8007561FF1208C7852261852262852263D272
:1013D800AF7522017524017525017526018560699F
:1013E800756A017888E6B40307C27D307602D27D3B
:1013F800D268D269753300120DFF120E301208E759
:101408001208EE1208E71208EE1208E7120B6E1225
:1014180006B0120C64120CAB1208EE120B5D306EA3
:10142800031206B12066031208033066031208335C
:10143800120C64120CDC1208EE120B6E306E0312E2
:1014480006ED120C64120D551208EE120B5D306E8B
:101458000312074B120C64120D861208EE120B6E63
:0F146800306E031207A8120C64120DFF1208EE6B
:1014770012084D120B5D120C64120E301208511235
:1014870008EE30692F856461856462856069756AD5
:101497000179187A0CC3E53399400CC269D26A8A7C
:1014A700357561FF0214BBC3E55C94014003021468
:1014B70014021549306A25206C22E535147006C2DE
:1014C7006AD26B8114F535C3E55C940140030214BD
:1014D700147888E6C39403600302154975360078CB
:1014E7008279A4E760027803C3E55F9850543074AB
:1014F70004E52A604D7888E6B40317207D05207639
:1015070007A119307602A119206C07D26C85646196
:10151700815378F0306C058564617820C3E5419884
:1015270050028114306C1BC26CC27D307602D27DB2
:10153700D26A75351285646181140536E55C6002EF
:10154700A14C753600C2AF120EAA7887E6FE760266
:10155700120F2B7887EEF6E4F522F523F524F5250F
:10156700F526F565752C00752D00D2AF1205A5126D
:101577000EAA78A4E66006C292C291C2903074099E
:10158700C3E5369404400201C541FD901A0D782049
:10159700121622E520B45A0CA3121622E520B4A590
:1015A700030215C0757CA5757DF1120EBF1215E0FB
:1015B700757C00757D000215DF901A0378807B0A21
:1015C700121622A308DBF9901A0F788C7B191216D2
:1015D70022A308DBF9901A2822C2AF121665121649
:1015E70042901A00740E121627A37409121627A325
:1015F7007415121627901A0378807B0A121626A3F1
:1016070008DBF9901A0F788C7B19121626A308DBD2
:10161700F9121678121656901A2822E493F622E643
:10162700438F01538FFDFFC3E583941C400122EFD5
:10163700857CB7857DB7F0538FFE22438F02438F9A
:1016470001857CB7857DB7901A0DF0538FFC2290EA
:101657001A0D745AD127901A0E74A5D127227A3001
:1016670079D07820901A40D122E520F709A3DAF73C
:10167700227A3079D0901A40E7D12709A3DAF922E4
:10168700AB74A875BB01027984BB02027985BB03E1
:10169700027986BB04027992BB05027987BB0602F1
:1016A70079A3BB0702799CBB08027988BB09027939
:1016B70089E8F7227C051205AADCFB22C2AF1205D6
:1016C700BA1205C11205C81205CF12059B1205BA39
:1016D7001205C11205C81205CF12059B1205BA12D1
:1016E70005C11205C81205CFD2AF22C2AF1205CF6E
:1016F7001205C81205C11205BA12059B1205CF12B1
:1017070005C81205C11205BA12059B1205CF1205AD
:10171700C81205C11205BAD2AF22AE74AF75C2AFF7
:101727001205BA1205BA1205BA12059BDEF21205A6
:10173700CF12059BDFF8D2AF22D1C3D1BBD1BB7586
:101747007401757501757600F1217C05AD5C120594
:10175700AAC3ED955C70F5C3E55C9401400AC3E547
:101767005C94FF403202177CD187B1E0D1C3C2AF8E
:1017770075EF16D1BBDCD50576C3E5769403500229
:1017870080C6D1BB0575E5741490009F93F808C314
:10179700E57598500280AED1BBD1BB0574C3E57423
:1017A700940A5002809C120EBFB1E0C2AF75EF16CB
:0217B700D1BBA4
:0319FD00021018BD
:101A00000E0915FFFFFFFF03040A0301015AA50198
:101A1000FFFFFFFFFF03FFFFFF25D0FAFA04FF01DE
:091A2000007AFF0101000300FF40
:101A400023484B696E67323041232020202020201C
:101A500023424C48454C4923463333302320202031
:101A60002020202020202020202020202020202076
:101C0000C2AFC2D353D9BF7581C043B20343FF8073
:101C1000752438752503B1DC7529A5752AF175E29F
:101C20004043F11053A4EF75D4FFD2847DFA7803BA
:101C300079E67C10752200752300901DE97B0675FE
:101C400024987525013084028145208408D8FBD969
:101C5000F9DCF781B7308408D8FBD9F9DCF781B714
:101C6000B19CE493A3C39A6004DDC381B7DBDBB10D
:101C70008E6002812E7B08E493FAA3B16FDBF87AC1
:101C800030B16F752200752300B18EEAFCEBFDC305
:101C9000ED94FE400EB18E8A278B28ED30E0048A49
:101CA000828B83B18E7AC270D8C3ED94FE601950D6
:101CB000CEBD002BEC600F7520007521FF7529004B
:101CC000752A000200008100A827A9280809D80465
:101CD000D90281DCB192EA89AAF281CE0D81A3C337
:101CE000ED94035053EDA2E092007AC5C3E58294CF
:101CF00000E583941C508A200010438F02438F011B
:101D00008529B7852AB7F0300029A827A92808090E
:101D1000438F01538FFDD804D902A133C3E58394C7
:101D20001C4003A3A11689AAE28529B7852AB7F02A
:101D3000A3A116538FFC817F7AC1BD030CE493A34A
:101D4000FAB153DCF8B14B817F8181AA22AB23B178
:101D50006FEBFAEA6222752608C3E52313F523E543
:101D60002213F52250066323A0632201D526EAB18F
:101D7000DCB1DC75260AEAF4200102D284300102CB
:101D8000C284B1DCC3134002C201D526EB22B1925A
:101D9000EAFB208402A192308402A197752608AE46
:101DA00024AF25C3EF13FFEE13FEB1E0B1DCC3EAAD
:101DB000133084024480FA30E703632201C3E52331
:101DC00013F523E52213F52250066323A0632201B5
:101DD000D526D9E52265236523F52222AE24AF2539
:101DE0000E0FDEFEDFFCD20122424C48656C6934E6
:071DF000373164F3300601F6
:00000001FF
